:100000000A128A113F2D00308A000408840A8207F0
:100010000034013400340A34003464340034E834E9
:1000200003341034273456345234313430346B3482
:100030003A34253464342034203443344434533443
:0E0040003A342534643420340D340A3400344C
:100A7E00B301B401B501B60183010A128A11AE2E7B
:100A8E00F20070088312031388000616720887009E
:100A9E00EF30F1007108860506160800F000572D9C
:100AAE0083160313981C5C2D5D2D572D5E2D70083B
:100ABE008312031399000800033083160313850075
:100ACE0001308600831203138601803083160313D0
:100ADE008700831203138701831603138801831281
:100AEE0003138801831603138901831203138901EB
:100AFE00203083160313980090308312031398004E
:100B0E00193083160313990020308C00E4308B00CB
:100B1E000530831203139F008030831603139F004A
:100B2E000800F00100300A128A1147250A128A11B4
:100B3E00F00101300A128A1147250A128A11F001BA
:100B4E0002300A128A1147250A128A11F001033067
:100B5E000A128A1147250A128A11F00104300A126C
:100B6E008A1147250A128A11F00105300A128A11DC
:100B7E0047250A128A11F00106300A128A114725FA
:100B8E000A128A11F00107300A128A1147250A1239
:100B9E008A110800790878040319D62DD72D0D2E49
:100BAE00FD010314FD0DE72D01300310F80DF90DB5
:100BBE00FF3E031DDC2D0130FC007C08FD07E72DF8
:100BCE00F91FEA2DEB2DDB2DED2DED2D79087B0296
:100BDE00031DF32D78087A02031CF62DF72DFE2D3A
:100BEE007808FA027908031CFB03FB02FE2D013084
:100BFE000310F90CF80CFF3E031DFF2D0130FD0212
:100C0E00031D0A2E0B2EED2D0D2E0D2E7B08F90138
:100C1E00F9077A08F801F807142E0800F600F70114
:100C2E00F801F401F501831603131F109F101F1115
:100C3E009F117608F20002300310F20DFF3E031DE5
:100C4E00232E0310720D3839831203139F001F14C5
:100C5E001F139F130D30F200F20B332E831203136A
:100C6E001F15392E1F1D3C2E3D2E392E3E2E1E08D1
:100C7E00F200F3017208F7007308F8007708F3002A
:100C8E00F2017208F7007308F800831603131E08AA
:100C9E00F200F3017208F7047308F80483120313C9
:100CAE000C137808F101F1077708F001F0075F2EB9
:100CBE000800F501F601710870040319672E682EFD
:100CCE00A62EF7010314F70D782E01300310F00D48
:100CDE00F10DFF3E031D6D2E0130F4007408F70771
:100CEE00782EF11F7B2E7C2E6C2E7E2E7E2E0130CA
:100CFE000310F50DF60DFF3E031D7F2E71087302D6
:100D0E00031D8B2E70087202031C8E2E8F2E972EB3
:100D1E007008F2027108031CF303F3027514972E88
:100D2E0001300310F10CF00CFF3E031D982E013024
:100D3E00F702031DA32EA42E7E2EA62EA62E760817
:100D4E00F101F1077508F001F007AD2E08000A1247
:100D5E008A1163250A128A110A128A1198250A121B
:100D6E008A11B92E83120313B101B201B101B2017E
:100D7E003208803AFF0080307F02031DC82E0230F9
:100D8E003102031CCB2ECC2ECE2EB92EB92E8312B1
:100D9E00031331080A128A1115260A128A118312B8
:100DAE0003133108B0003007333E840070088313FC
:100DBE008000840A710880003408A101A10733085D
:100DCE00A001A0073608A301A3073508A201A207B8
:100DDE000B300A128A1110270A128A11013083125F
:100DEE000313B1070318B20A0030B2073208803A73
:100DFE00FF0080307F02031D062F02303102031CDC
:100E0E00092F0A2FCE2EB92EB92EB92E0A128A11FB
:100E1E00002883120313A9002030A4002408A70081
:100E2E00E92F2F08253A03191D2F1E2F252F2F08C6
:100E3E000A128A1155250A128A11E92FA8012C2FA0
:100E4E00FF2F412F412FE92F412F0130A907FF30EE
:100E5E00290784000A128A1103200A128A11AF0090
:100E6E00003A0319FF2F643A0319412F0D3A031963
:100E7E00412FE92F2708840083130008AB00840A52
:100E8E000008AC000230A4002408A707AC1F502FA6
:100E9E00512F5B2F0330A4002408A804AB09AC0922
:100EAE00AB0A0319AC0A5B2FAF010314AF0D2F0869
:100EBE00053A031D632F642F662F8E2F8E2F2F085A
:100ECE00A4002407013E84000A128A1103200A128C
:100EDE008A11A5000A128A1103200A128A11A6008D
:100EEE0026082C02031D7D2F25082B020318802FA8
:100EFE00812F832F8E2F8E2F0130A4002408AF0751
:100F0E002F08053A031D8C2F8D2F662F8E2F280844
:100F1E0003390319932F942F9B2F2D300A128A1108
:100F2E0055250A128A119B2F831203132F08A40032
:100F3E002408AA00DB2F0A30F8000030F9002A0836
:100F4E00A4002407013E84000A128A1103200A120B
:100F5E008A11F0000A128A1103200A128A11F10076
:100F6E002C08F301F3072B08F201F2070A128A117B
:100F7E0060260A128A117108FB01FB077008FA013C
:100F8E00FA070A128A11D1250A128A117808303E00
:100F9E0083120313A5002508AF002F080A128A1129
:100FAE0055250A128A11DB2FFF3083120313A4007A
:100FBE002408AA072A08FF3A031DE62FE72FA22FBF
:100FCE00E92FE92F013083120313A907FF302907F8
:100FDE0084000A128A1103200A128A11A40024081E
:100FEE00AF00AF08031DFC2FFD2F182FFF2FFF2F73
:020FFE000800E9
:00000001FF
